 setlocal001

 Timestamp is 39a6233e (reproducible build file hash)

 Preferred load address is 0000000180000000

 Start         Length     Name                   Class
 0001:00000000 000034b0H .text$mn                CODE
 0001:000034b0 00000036H .text$mn$00             CODE
 0001:000034e6 00000092H .text$x                 CODE
 0002:00000000 00000198H .idata$5                DATA
 0002:00000198 00000038H .00cfg                  DATA
 0002:000001d0 00000008H .CRT$XCA                DATA
 0002:000001d8 00000008H .CRT$XCZ                DATA
 0002:000001e0 00000008H .CRT$XIA                DATA
 0002:000001e8 00000008H .CRT$XIC                DATA
 0002:000001f0 00000008H .CRT$XIZ                DATA
 0002:000001f8 00000008H .CRT$XLA                DATA
 0002:00000200 00000008H .CRT$XLZ                DATA
 0002:00000208 00000008H .CRT$XPA                DATA
 0002:00000210 00000008H .CRT$XPZ                DATA
 0002:00000218 00000008H .CRT$XTA                DATA
 0002:00000220 00000010H .CRT$XTZ                DATA
 0002:00000228 00000000H .gehcont$y              DATA
 0002:00000228 00000000H .gfids$y                DATA
 0002:00000230 00001e50H .rdata                  DATA
 0002:00002080 00000000H .rdata$CastGuardVftablesA DATA
 0002:00002080 00000000H .rdata$CastGuardVftablesC DATA
 0002:00002080 00000028H .rdata$T                DATA
 0002:000020a8 000000a4H .rdata$voltmd           DATA
 0002:0000214c 0000031cH .rdata$zzzdbg           DATA
 0002:00002468 00000008H .rtc$IAA                DATA
 0002:00002470 00000008H .rtc$IZZ                DATA
 0002:00002478 00000008H .rtc$TAA                DATA
 0002:00002480 00000008H .rtc$TZZ                DATA
 0002:00002488 00000004H .tls                    DATA
 0002:0000248c 00000004H .tls$                   DATA
 0002:00002490 00000008H .tls$ZZZ                DATA
 0002:00002498 00000318H .xdata                  DATA
 0002:000027b0 000003e4H .edata                  DATA
 0002:00002b94 00000064H .idata$2                DATA
 0002:00002bf8 00000018H .idata$3                DATA
 0002:00002c10 00000198H .idata$4                DATA
 0002:00002da8 0000041eH .idata$6                DATA
 0003:00000000 00000080H .data                   DATA
 0003:00000080 0001b3b8H .bss                    DATA
 0004:00000000 00000390H .pdata                  DATA

  Address         Publics by Value              Rva+Base               Lib:Object

 0000:00000000       __AbsoluteZero             0000000000000000     <absolute>
 0000:00000000       ___safe_se_handler_count   0000000000000000     <absolute>
 0000:00000000       ___safe_se_handler_table   0000000000000000     <absolute>
 0000:00000000       __arm64x_extra_rfe_table   0000000000000000     <absolute>
 0000:00000000       __arm64x_extra_rfe_table_size 0000000000000000     <absolute>
 0000:00000000       __arm64x_native_entrypoint 0000000000000000     <absolute>
 0000:00000000       __arm64x_redirection_metadata 0000000000000000     <absolute>
 0000:00000000       __arm64x_redirection_metadata_count 0000000000000000     <absolute>
 0000:00000000       __dynamic_value_reloc_table 0000000000000000     <absolute>
 0000:00000000       __enclave_config           0000000000000000     <absolute>
 0000:00000000       __guard_check_icall_a64n_fptr 0000000000000000     <absolute>
 0000:00000000       __guard_eh_cont_count      0000000000000000     <absolute>
 0000:00000000       __guard_eh_cont_table      0000000000000000     <absolute>
 0000:00000000       __guard_fids_count         0000000000000000     <absolute>
 0000:00000000       __guard_fids_table         0000000000000000     <absolute>
 0000:00000000       __guard_iat_count          0000000000000000     <absolute>
 0000:00000000       __guard_iat_table          0000000000000000     <absolute>
 0000:00000000       __guard_longjmp_count      0000000000000000     <absolute>
 0000:00000000       __guard_longjmp_table      0000000000000000     <absolute>
 0000:00000000       __hybrid_auxiliary_iat     0000000000000000     <absolute>
 0000:00000000       __hybrid_auxiliary_iat_copy 0000000000000000     <absolute>
 0000:00000000       __hybrid_code_map          0000000000000000     <absolute>
 0000:00000000       __hybrid_code_map_count    0000000000000000     <absolute>
 0000:00000000       __x64_code_ranges_to_entry_points 0000000000000000     <absolute>
 0000:00000000       __x64_code_ranges_to_entry_points_count 0000000000000000     <absolute>
 0000:00000100       __guard_flags              0000000000000100     <absolute>
 0000:00000000       __ImageBase                0000000180000000     <linker-defined>
 0001:00000000       ?NewObject@JNIEnv_@@QEAAPEAV_jobject@@PEAV_jclass@@PEAU_jmethodID@@ZZ 0000000180001000 f i libsetlocal001.obj
 0001:00000028       ?SetEventNotificationMode@_jvmtiEnv@@QEAA?AW4jvmtiError@@W4jvmtiEventMode@@W4jvmtiEvent@@PEAV_jobject@@ZZ 0000000180001028 f i libsetlocal001.obj
 0001:00000034       ?TranslateError@@YAPEBDW4jvmtiError@@@Z 0000000180001034 f   libsetlocal001.obj
 0001:000002ec       ?nsk_jni_check_exception@@YAHPEAUJNIEnv_@@QEBDH@Z 00000001800012ec f   libsetlocal001.obj
 0001:00000430       ?nsk_jni_lverify@@YAHHPEAUJNIEnv_@@HQEBDH1ZZ 0000000180001430 f   libsetlocal001.obj
 0001:000004d0       Agent_Initialize           00000001800014d0 f   libsetlocal001.obj
 0001:00000628       Agent_OnAttach             0000000180001628 f   libsetlocal001.obj
 0001:00000628       Agent_OnLoad               0000000180001628 f   libsetlocal001.obj
 0001:00000630       Breakpoint                 0000000180001630 f   libsetlocal001.obj
 0001:00000dd4       Java_nsk_jvmti_SetLocalVariable_setlocal001_getMethReady 0000000180001dd4 f   libsetlocal001.obj
 0001:00000ff4       Java_nsk_jvmti_SetLocalVariable_setlocal001_getRes 0000000180001ff4 f   libsetlocal001.obj
 0001:00000ffc       Java_nsk_jvmti_unit_FollowReferences_FollowRefObjects_addRefToVerify 0000000180001ffc f   libsetlocal001.obj
 0001:000011d4       Java_nsk_jvmti_unit_FollowReferences_FollowRefObjects_getTag 00000001800021d4 f   libsetlocal001.obj
 0001:00001294       Java_nsk_jvmti_unit_FollowReferences_FollowRefObjects_resetRefsToVerify 0000000180002294 f   libsetlocal001.obj
 0001:0000129c       Java_nsk_jvmti_unit_FollowReferences_FollowRefObjects_resetTags 000000018000229c f   libsetlocal001.obj
 0001:000012e0       Java_nsk_jvmti_unit_FollowReferences_FollowRefObjects_setTag 00000001800022e0 f   libsetlocal001.obj
 0001:00001538       Java_nsk_share_jvmti_ArgumentHandler_getAgentOptionsString 0000000180002538 f   libsetlocal001.obj
 0001:000015e8       Java_nsk_share_jvmti_DebugeeClass_checkStatus 00000001800025e8 f   libsetlocal001.obj
 0001:00001670       Java_nsk_share_jvmti_DebugeeClass_resetAgentData 0000000180002670 f   libsetlocal001.obj
 0001:000016d0       Java_nsk_share_jvmti_RedefineAgent_agentStatus 00000001800026d0 f   libsetlocal001.obj
 0001:000016dc       Java_nsk_share_jvmti_RedefineAgent_isRedefined 00000001800026dc f   libsetlocal001.obj
 0001:000016e8       Java_nsk_share_jvmti_RedefineAgent_redefineAttempted 00000001800026e8 f   libsetlocal001.obj
 0001:000016f4       MA_checkStatus             00000001800026f4 f   libsetlocal001.obj
 0001:00001798       __local_stdio_printf_options 0000000180002798 f i libsetlocal001.obj
 0001:000019c4       exitOnError                00000001800029c4 f   libsetlocal001.obj
 0001:00001a78       fprintf                    0000000180002a78 f i libsetlocal001.obj
 0001:00001abc       nsk_jvmti_lverify          0000000180002abc f   libsetlocal001.obj
 0001:00001bac       nsk_jvmti_resetAgentData   0000000180002bac f   libsetlocal001.obj
 0001:00001c2c       nsk_jvmti_setFailStatus    0000000180002c2c f   libsetlocal001.obj
 0001:00001c68       nsk_lcomplain              0000000180002c68 f   libsetlocal001.obj
 0001:00001c88       nsk_ldisplay               0000000180002c88 f   libsetlocal001.obj
 0001:00001ca8       nsk_ltrace                 0000000180002ca8 f   libsetlocal001.obj
 0001:00001cc8       nsk_lvcomplain             0000000180002cc8 f   libsetlocal001.obj
 0001:00001e80       nsk_lvdisplay              0000000180002e80 f   libsetlocal001.obj
 0001:00001ecc       nsk_lverify                0000000180002ecc f   libsetlocal001.obj
 0001:00001f28       nsk_lvtrace                0000000180002f28 f   libsetlocal001.obj
 0001:00001f88       nsk_printf                 0000000180002f88 f   libsetlocal001.obj
 0001:00001fb0       nsk_vprintf                0000000180002fb0 f   libsetlocal001.obj
 0001:00002064       printf                     0000000180003064 f i libsetlocal001.obj
 0001:0000258c       __raise_securityfailure    000000018000358c f   MSVCRT:gs_report.obj
 0001:000025c0       __report_gsfailure         00000001800035c0 f   MSVCRT:gs_report.obj
 0001:00002800       __GSHandlerCheck           0000000180003800 f   MSVCRT:gshandler.obj
 0001:00002820       __GSHandlerCheckCommon     0000000180003820 f   MSVCRT:gshandler.obj
 0001:00002890       __security_check_cookie    0000000180003890 f   MSVCRT:amdsecgs.obj
 0001:00002bd0       _DllMainCRTStartup         0000000180003bd0 f   MSVCRT:dll_dllmain.obj
 0001:00002c10       __scrt_acquire_startup_lock 0000000180003c10 f   MSVCRT:utility.obj
 0001:00002c4c       __scrt_dllmain_after_initialize_c 0000000180003c4c f   MSVCRT:utility.obj
 0001:00002c80       __scrt_dllmain_before_initialize_c 0000000180003c80 f   MSVCRT:utility.obj
 0001:00002c98       __scrt_dllmain_crt_thread_attach 0000000180003c98 f   MSVCRT:utility.obj
 0001:00002cc0       __scrt_dllmain_crt_thread_detach 0000000180003cc0 f   MSVCRT:utility.obj
 0001:00002cd8       __scrt_dllmain_exception_filter 0000000180003cd8 f   MSVCRT:utility.obj
 0001:00002d38       __scrt_dllmain_uninitialize_c 0000000180003d38 f   MSVCRT:utility.obj
 0001:00002d68       __scrt_dllmain_uninitialize_critical 0000000180003d68 f   MSVCRT:utility.obj
 0001:00002d7c       __scrt_initialize_crt      0000000180003d7c f   MSVCRT:utility.obj
 0001:00002dc8       __scrt_initialize_onexit_tables 0000000180003dc8 f   MSVCRT:utility.obj
 0001:00002e54       __scrt_is_nonwritable_in_current_image 0000000180003e54 f   MSVCRT:utility.obj
 0001:00002eec       __scrt_release_startup_lock 0000000180003eec f   MSVCRT:utility.obj
 0001:00002f10       __scrt_uninitialize_crt    0000000180003f10 f   MSVCRT:utility.obj
 0001:00002f3c       _onexit                    0000000180003f3c f   MSVCRT:utility.obj
 0001:00002f78       atexit                     0000000180003f78 f   MSVCRT:utility.obj
 0001:00002f90       __crt_debugger_hook        0000000180003f90 f   MSVCRT:utility_desktop.obj
 0001:00002f98       __scrt_fastfail            0000000180003f98 f   MSVCRT:utility_desktop.obj
 0001:000030e4       _guard_check_icall_nop     00000001800040e4 f i MSVCRT:guard_support.obj
 0001:000030e8       __security_init_cookie     00000001800040e8 f   MSVCRT:gs_support.obj
 0001:00003194       DllMain                    0000000180004194 f   MSVCRT:dll_dllmain_stub.obj
 0001:000031b8       ?__scrt_initialize_type_info@@YAXXZ 00000001800041b8 f   MSVCRT:tncleanup.obj
 0001:000031c8       ?__scrt_uninitialize_type_info@@YAXXZ 00000001800041c8 f   MSVCRT:tncleanup.obj
 0001:000031d4       __local_stdio_scanf_options 00000001800041d4 f i MSVCRT:default_local_stdio_options.obj
 0001:000031dc       __scrt_initialize_default_local_stdio_options 00000001800041dc f   MSVCRT:default_local_stdio_options.obj
 0001:000031f8       __scrt_get_dyn_tls_init_callback 00000001800041f8 f   MSVCRT:dyn_tls_init.obj
 0001:00003200       _RTC_Initialize            0000000180004200 f   MSVCRT:initsect.obj
 0001:0000323c       _RTC_Terminate             000000018000423c f   MSVCRT:initsect.obj
 0001:00003278       __isa_available_init       0000000180004278 f   MSVCRT:cpu_disp.obj
 0001:00003424       _get_startup_argv_mode     0000000180004424 f   MSVCRT:argv_mode.obj
 0001:0000342c       __scrt_is_ucrt_dll_in_use  000000018000442c f   MSVCRT:ucrt_detection.obj
 0001:00003440       memcpy                     0000000180004440 f   vcruntime:VCRUNTIME140.dll
 0001:00003446       memset                     0000000180004446 f   vcruntime:VCRUNTIME140.dll
 0001:0000344c       strchr                     000000018000444c f   vcruntime:VCRUNTIME140.dll
 0001:00003452       __C_specific_handler       0000000180004452 f   vcruntime:VCRUNTIME140.dll
 0001:00003458       __std_type_info_destroy_list 0000000180004458 f   vcruntime:VCRUNTIME140.dll
 0001:0000345e       strcmp                     000000018000445e f   ucrt:api-ms-win-crt-string-l1-1-0.dll
 0001:00003464       strlen                     0000000180004464 f   ucrt:api-ms-win-crt-string-l1-1-0.dll
 0001:0000346a       _initterm                  000000018000446a f   ucrt:api-ms-win-crt-runtime-l1-1-0.dll
 0001:00003470       _initterm_e                0000000180004470 f   ucrt:api-ms-win-crt-runtime-l1-1-0.dll
 0001:00003476       _seh_filter_dll            0000000180004476 f   ucrt:api-ms-win-crt-runtime-l1-1-0.dll
 0001:0000347c       _configure_narrow_argv     000000018000447c f   ucrt:api-ms-win-crt-runtime-l1-1-0.dll
 0001:00003482       _initialize_narrow_environment 0000000180004482 f   ucrt:api-ms-win-crt-runtime-l1-1-0.dll
 0001:00003488       _initialize_onexit_table   0000000180004488 f   ucrt:api-ms-win-crt-runtime-l1-1-0.dll
 0001:0000348e       _register_onexit_function  000000018000448e f   ucrt:api-ms-win-crt-runtime-l1-1-0.dll
 0001:00003494       _execute_onexit_table      0000000180004494 f   ucrt:api-ms-win-crt-runtime-l1-1-0.dll
 0001:0000349a       _crt_atexit                000000018000449a f   ucrt:api-ms-win-crt-runtime-l1-1-0.dll
 0001:000034a0       _cexit                     00000001800044a0 f   ucrt:api-ms-win-crt-runtime-l1-1-0.dll
 0001:000034a8       __acrt_initialize          00000001800044a8 f   MSVCRT:ucrt_stubs.obj
 0001:000034a8       __acrt_thread_attach       00000001800044a8 f   MSVCRT:ucrt_stubs.obj
 0001:000034a8       __acrt_thread_detach       00000001800044a8 f   MSVCRT:ucrt_stubs.obj
 0001:000034a8       __acrt_uninitialize        00000001800044a8 f   MSVCRT:ucrt_stubs.obj
 0001:000034a8       __acrt_uninitialize_critical 00000001800044a8 f   MSVCRT:ucrt_stubs.obj
 0001:000034a8       __scrt_stub_for_acrt_initialize 00000001800044a8 f   MSVCRT:ucrt_stubs.obj
 0001:000034a8       __scrt_stub_for_acrt_thread_attach 00000001800044a8 f   MSVCRT:ucrt_stubs.obj
 0001:000034a8       __scrt_stub_for_acrt_thread_detach 00000001800044a8 f   MSVCRT:ucrt_stubs.obj
 0001:000034a8       __scrt_stub_for_acrt_uninitialize 00000001800044a8 f   MSVCRT:ucrt_stubs.obj
 0001:000034a8       __scrt_stub_for_acrt_uninitialize_critical 00000001800044a8 f   MSVCRT:ucrt_stubs.obj
 0001:000034a8       __vcrt_initialize          00000001800044a8 f   MSVCRT:ucrt_stubs.obj
 0001:000034a8       __vcrt_thread_attach       00000001800044a8 f   MSVCRT:ucrt_stubs.obj
 0001:000034a8       __vcrt_thread_detach       00000001800044a8 f   MSVCRT:ucrt_stubs.obj
 0001:000034a8       __vcrt_uninitialize        00000001800044a8 f   MSVCRT:ucrt_stubs.obj
 0001:000034a8       __vcrt_uninitialize_critical 00000001800044a8 f   MSVCRT:ucrt_stubs.obj
 0001:000034ac       __scrt_stub_for_is_c_termination_complete 00000001800044ac f   MSVCRT:ucrt_stubs.obj
 0001:000034ac       _is_c_termination_complete 00000001800044ac f   MSVCRT:ucrt_stubs.obj
 0001:000034c0       _guard_dispatch_icall_nop  00000001800044c0 f   MSVCRT:guard_dispatch.obj
 0001:000034e0       _guard_xfg_dispatch_icall_nop 00000001800044e0 f   MSVCRT:guard_xfg_dispatch.obj
 0002:00000000       __imp_RtlCaptureContext    0000000180005000     kernel32:KERNEL32.dll
 0002:00000008       __imp_RtlLookupFunctionEntry 0000000180005008     kernel32:KERNEL32.dll
 0002:00000010       __imp_RtlVirtualUnwind     0000000180005010     kernel32:KERNEL32.dll
 0002:00000018       __imp_UnhandledExceptionFilter 0000000180005018     kernel32:KERNEL32.dll
 0002:00000020       __imp_SetUnhandledExceptionFilter 0000000180005020     kernel32:KERNEL32.dll
 0002:00000028       __imp_GetCurrentProcess    0000000180005028     kernel32:KERNEL32.dll
 0002:00000030       __imp_TerminateProcess     0000000180005030     kernel32:KERNEL32.dll
 0002:00000038       __imp_IsProcessorFeaturePresent 0000000180005038     kernel32:KERNEL32.dll
 0002:00000040       __imp_CloseHandle          0000000180005040     kernel32:KERNEL32.dll
 0002:00000048       __imp_InitializeCriticalSectionAndSpinCount 0000000180005048     kernel32:KERNEL32.dll
 0002:00000050       __imp_DeleteCriticalSection 0000000180005050     kernel32:KERNEL32.dll
 0002:00000058       __imp_CreateEventW         0000000180005058     kernel32:KERNEL32.dll
 0002:00000060       __imp_GetModuleHandleW     0000000180005060     kernel32:KERNEL32.dll
 0002:00000068       __imp_GetProcAddress       0000000180005068     kernel32:KERNEL32.dll
 0002:00000070       __imp_IsDebuggerPresent    0000000180005070     kernel32:KERNEL32.dll
 0002:00000078       __imp_QueryPerformanceCounter 0000000180005078     kernel32:KERNEL32.dll
 0002:00000080       __imp_GetCurrentProcessId  0000000180005080     kernel32:KERNEL32.dll
 0002:00000088       __imp_GetCurrentThreadId   0000000180005088     kernel32:KERNEL32.dll
 0002:00000090       __imp_GetSystemTimeAsFileTime 0000000180005090     kernel32:KERNEL32.dll
 0002:00000098       __imp_DisableThreadLibraryCalls 0000000180005098     kernel32:KERNEL32.dll
 0002:000000a0       __imp_InitializeSListHead  00000001800050a0     kernel32:KERNEL32.dll
 0002:000000a8       \177KERNEL32_NULL_THUNK_DATA 00000001800050a8     kernel32:KERNEL32.dll
 0002:000000b0       __imp_memcpy               00000001800050b0     vcruntime:VCRUNTIME140.dll
 0002:000000b8       __imp_memset               00000001800050b8     vcruntime:VCRUNTIME140.dll
 0002:000000c0       __imp_strchr               00000001800050c0     vcruntime:VCRUNTIME140.dll
 0002:000000c8       __imp___C_specific_handler 00000001800050c8     vcruntime:VCRUNTIME140.dll
 0002:000000d0       __imp___std_type_info_destroy_list 00000001800050d0     vcruntime:VCRUNTIME140.dll
 0002:000000d8       \177VCRUNTIME140_NULL_THUNK_DATA 00000001800050d8     vcruntime:VCRUNTIME140.dll
 0002:000000e0       __imp__errno               00000001800050e0     ucrt:api-ms-win-crt-runtime-l1-1-0.dll
 0002:000000e8       __imp_exit                 00000001800050e8     ucrt:api-ms-win-crt-runtime-l1-1-0.dll
 0002:000000f0       __imp__cexit               00000001800050f0     ucrt:api-ms-win-crt-runtime-l1-1-0.dll
 0002:000000f8       __imp__crt_atexit          00000001800050f8     ucrt:api-ms-win-crt-runtime-l1-1-0.dll
 0002:00000100       __imp__execute_onexit_table 0000000180005100     ucrt:api-ms-win-crt-runtime-l1-1-0.dll
 0002:00000108       __imp__register_onexit_function 0000000180005108     ucrt:api-ms-win-crt-runtime-l1-1-0.dll
 0002:00000110       __imp__initialize_onexit_table 0000000180005110     ucrt:api-ms-win-crt-runtime-l1-1-0.dll
 0002:00000118       __imp__initialize_narrow_environment 0000000180005118     ucrt:api-ms-win-crt-runtime-l1-1-0.dll
 0002:00000120       __imp__configure_narrow_argv 0000000180005120     ucrt:api-ms-win-crt-runtime-l1-1-0.dll
 0002:00000128       __imp__seh_filter_dll      0000000180005128     ucrt:api-ms-win-crt-runtime-l1-1-0.dll
 0002:00000130       __imp__initterm_e          0000000180005130     ucrt:api-ms-win-crt-runtime-l1-1-0.dll
 0002:00000138       __imp__initterm            0000000180005138     ucrt:api-ms-win-crt-runtime-l1-1-0.dll
 0002:00000140       \177api-ms-win-crt-runtime-l1-1-0_NULL_THUNK_DATA 0000000180005140     ucrt:api-ms-win-crt-runtime-l1-1-0.dll
 0002:00000148       __imp___acrt_iob_func      0000000180005148     ucrt:api-ms-win-crt-stdio-l1-1-0.dll
 0002:00000150       __imp_fflush               0000000180005150     ucrt:api-ms-win-crt-stdio-l1-1-0.dll
 0002:00000158       __imp___stdio_common_vsprintf 0000000180005158     ucrt:api-ms-win-crt-stdio-l1-1-0.dll
 0002:00000160       __imp___stdio_common_vfprintf 0000000180005160     ucrt:api-ms-win-crt-stdio-l1-1-0.dll
 0002:00000168       \177api-ms-win-crt-stdio-l1-1-0_NULL_THUNK_DATA 0000000180005168     ucrt:api-ms-win-crt-stdio-l1-1-0.dll
 0002:00000170       __imp_strcmp               0000000180005170     ucrt:api-ms-win-crt-string-l1-1-0.dll
 0002:00000178       __imp__strdup              0000000180005178     ucrt:api-ms-win-crt-string-l1-1-0.dll
 0002:00000178       __imp_strdup               0000000180005178     ucrt:api-ms-win-crt-string-l1-1-0.dll
 0002:00000180       __imp_strlen               0000000180005180     ucrt:api-ms-win-crt-string-l1-1-0.dll
 0002:00000188       __imp_strncpy              0000000180005188     ucrt:api-ms-win-crt-string-l1-1-0.dll
 0002:00000190       \177api-ms-win-crt-string-l1-1-0_NULL_THUNK_DATA 0000000180005190     ucrt:api-ms-win-crt-string-l1-1-0.dll
 0002:00000198       __guard_check_icall_fptr   0000000180005198     MSVCRT:guard_support.obj
 0002:000001a0       __guard_xfg_check_icall_fptr 00000001800051a0     MSVCRT:guard_support.obj
 0002:000001a8       __guard_dispatch_icall_fptr 00000001800051a8     MSVCRT:guard_support.obj
 0002:000001b0       __guard_xfg_dispatch_icall_fptr 00000001800051b0     MSVCRT:guard_support.obj
 0002:000001b8       __guard_xfg_table_dispatch_icall_fptr 00000001800051b8     MSVCRT:guard_support.obj
 0002:000001c0       __castguard_check_failure_os_handled_fptr 00000001800051c0     MSVCRT:guard_support.obj
 0002:000001c8       __guard_memcpy_fptr        00000001800051c8     vcruntime:softmemtag.obj
 0002:000001d0       __xc_a                     00000001800051d0     MSVCRT:initializers.obj
 0002:000001d8       __xc_z                     00000001800051d8     MSVCRT:initializers.obj
 0002:000001e0       __xi_a                     00000001800051e0     MSVCRT:initializers.obj
 0002:000001f0       __xi_z                     00000001800051f0     MSVCRT:initializers.obj
 0002:000001f8       __xl_a                     00000001800051f8     MSVCRT:tlssup.obj
 0002:00000200       __xl_z                     0000000180005200     MSVCRT:tlssup.obj
 0002:00000208       __xp_a                     0000000180005208     MSVCRT:initializers.obj
 0002:00000210       __xp_z                     0000000180005210     MSVCRT:initializers.obj
 0002:00000218       __xt_a                     0000000180005218     MSVCRT:initializers.obj
 0002:00000220       __xt_z                     0000000180005220     MSVCRT:initializers.obj
 0002:00000230       g_refKindStr               0000000180005230     libsetlocal001.obj
 0002:000003e0       ??_C@_09BPLDFGCI@unknown_0@ 00000001800053e0     libsetlocal001.obj
 0002:000003f0       ??_C@_0BL@FPNMECJD@JVMTI_HEAP_REFERENCE_CLASS@ 00000001800053f0     libsetlocal001.obj
 0002:00000410       ??_C@_0BL@FKGKKLNM@JVMTI_HEAP_REFERENCE_FIELD@ 0000000180005410     libsetlocal001.obj
 0002:00000430       ??_C@_0CD@CAEHCFJF@JVMTI_HEAP_REFERENCE_ARRAY_ELEM@ 0000000180005430     libsetlocal001.obj
 0002:00000458       ??_C@_0CC@DNEBMCNK@JVMTI_HEAP_REFERENCE_CLASS_LOAD@ 0000000180005458     libsetlocal001.obj
 0002:00000480       ??_C@_0BN@CJMIPEBB@JVMTI_HEAP_REFERENCE_SIGNERS@ 0000000180005480     libsetlocal001.obj
 0002:000004a0       ??_C@_0CH@HBOIDPEB@JVMTI_HEAP_REFERENCE_PROTECTION@ 00000001800054a0     libsetlocal001.obj
 0002:000004c8       ??_C@_0BP@MDKGDGKL@JVMTI_HEAP_REFERENCE_INTERFACE@ 00000001800054c8     libsetlocal001.obj
 0002:000004e8       ??_C@_0CC@JJMIHNJH@JVMTI_HEAP_REFERENCE_STATIC_FIE@ 00000001800054e8     libsetlocal001.obj
 0002:00000510       ??_C@_0CD@IDHEEGID@JVMTI_HEAP_REFERENCE_CONSTANT_P@ 0000000180005510     libsetlocal001.obj
 0002:00000538       ??_C@_0CA@EFFCHNG@JVMTI_HEAP_REFERENCE_SUPERCLASS@ 0000000180005538     libsetlocal001.obj
 0002:00000558       ??_C@_0L@PCDFHGCJ@unknown_11@ 0000000180005558     libsetlocal001.obj
 0002:00000568       ??_C@_0L@NJBICFOK@unknown_12@ 0000000180005568     libsetlocal001.obj
 0002:00000578       ??_C@_0L@MAADBEKL@unknown_13@ 0000000180005578     libsetlocal001.obj
 0002:00000588       ??_C@_0L@IPECICGM@unknown_14@ 0000000180005588     libsetlocal001.obj
 0002:00000598       ??_C@_0L@JGFJLDCN@unknown_15@ 0000000180005598     libsetlocal001.obj
 0002:000005a8       ??_C@_0L@LNHEOAOO@unknown_16@ 00000001800055a8     libsetlocal001.obj
 0002:000005b8       ??_C@_0L@KEGPNBKP@unknown_17@ 00000001800055b8     libsetlocal001.obj
 0002:000005c8       ??_C@_0L@CDPHMNGA@unknown_18@ 00000001800055c8     libsetlocal001.obj
 0002:000005d8       ??_C@_0L@DKOMPMCB@unknown_19@ 00000001800055d8     libsetlocal001.obj
 0002:000005e8       ??_C@_0L@OJGIPJDB@unknown_20@ 00000001800055e8     libsetlocal001.obj
 0002:000005f8       ??_C@_0CA@KAOFNDEM@JVMTI_HEAP_REFERENCE_JNI_GLOBAL@ 00000001800055f8     libsetlocal001.obj
 0002:00000618       ??_C@_0CC@HPFAJBK@JVMTI_HEAP_REFERENCE_SYSTEM_CLA@ 0000000180005618     libsetlocal001.obj
 0002:00000640       ??_C@_0BN@FDEGFOHC@JVMTI_HEAP_REFERENCE_MONITOR@ 0000000180005640     libsetlocal001.obj
 0002:00000660       ??_C@_0CB@HKIBCMAJ@JVMTI_HEAP_REFERENCE_STACK_LOCA@ 0000000180005660     libsetlocal001.obj
 0002:00000688       ??_C@_0BP@EAACMMOE@JVMTI_HEAP_REFERENCE_JNI_LOCAL@ 0000000180005688     libsetlocal001.obj
 0002:000006a8       ??_C@_0BM@IJDEOGOE@JVMTI_HEAP_REFERENCE_THREAD@ 00000001800056a8     libsetlocal001.obj
 0002:000006c8       ??_C@_0BL@EDGPPKC@JVMTI_HEAP_REFERENCE_OTHER@ 00000001800056c8     libsetlocal001.obj
 0002:000006e4       ??_C@_04BCJPDBDA@Code@     00000001800056e4     libsetlocal001.obj
 0002:000006f0       ??_C@_0BA@OCLMCFKC@LineNumberTable@ 00000001800056f0     libsetlocal001.obj
 0002:00000700       ??_C@_0BD@CPAEPILC@LocalVariableTable@ 0000000180005700     libsetlocal001.obj
 0002:00000718       ??_C@_0BH@NMBDNHBD@LocalVariableTypeTable@ 0000000180005718     libsetlocal001.obj
 0002:00000730       ??_C@_0O@HIHEEDNJ@StackMapTable@ 0000000180005730     libsetlocal001.obj
 0002:00000740       ??_C@_0L@HCDIAMJG@?9?5?$CFs?0?5?$CFd?3?5@ 0000000180005740     libsetlocal001.obj
 0002:00000750       ??_C@_0JI@HLPECLFI@?$CD?5?4?4?4?6?$CD?5ERROR?3?5too?5many?5complai@ 0000000180005750     libsetlocal001.obj
 0002:000007f0       ??_C@_0ED@JNEKCCOB@The?5following?5fake?5exception?5st@ 00000001800057f0     libsetlocal001.obj
 0002:00000838       ??_C@_0CN@FCNMDFBH@nsk?4share?4Fake_Exception_for_RU@ 0000000180005838     libsetlocal001.obj
 0002:00000868       ??_C@_08PGFFNAEI@?$CI?$CFs?3?$CFd?$CJ?5@ 0000000180005868     libsetlocal001.obj
 0002:00000878       ??_C@_0DP@IENMAEGI@s?2test?2hotspot?2jtreg?2vmTestbase@ 0000000180005878     libsetlocal001.obj
 0002:000008b8       ??_C@_0BL@NDJLFFJB@?7at?5nsk_lvcomplain?$CI?$CFs?3?$CFd?$CJ?6@ 00000001800058b8     libsetlocal001.obj
 0002:000008d8       ??_C@_0BC@JOOKAFKF@?$CD?5ERROR?3?5?$CFs?0?5?$CFd?3?5@ 00000001800058d8     libsetlocal001.obj
 0002:000008f0       ??_C@_09KJEAHMEH@?$CD?5ERROR?3?5@ 00000001800058f0     libsetlocal001.obj
 0002:000008fc       ??_C@_02GPIOPFAK@?$DO?$DO@ 00000001800058fc     libsetlocal001.obj
 0002:00000900       ??_C@_02FODMEDOG@?$DM?$DM@ 0000000180005900     libsetlocal001.obj
 0002:00000904       ??_C@_02DJGKEECL@?4?4@     0000000180005904     libsetlocal001.obj
 0002:00000908       ??_C@_0O@CJPGJOAF@?9?5?$CFs?0?5?$CFd?3?5?$CFs?5@ 0000000180005908     libsetlocal001.obj
 0002:00000918       ??_C@_0CB@IAKPDOIC@?$CD?5?5?5verified?5assertion?5is?5FALSE@ 0000000180005918     libsetlocal001.obj
 0002:00000940       ??_C@_0CO@LGONDEPD@stdout?3?5fflush?5failed?5?9?5err?$DN?$CFd?5@ 0000000180005940     libsetlocal001.obj
 0002:00000970       ??_C@_0CO@KBGKJPBD@stderr?3?5fflush?5failed?5?9?5err?$DN?$CFd?5@ 0000000180005970     libsetlocal001.obj
 0002:000009a0       ??_C@_0BB@JCNMKLLK@JVMTI_ERROR_NONE@ 00000001800059a0     libsetlocal001.obj
 0002:000009b8       ??_C@_0BL@LDIMKLPH@JVMTI_ERROR_INVALID_THREAD@ 00000001800059b8     libsetlocal001.obj
 0002:000009d8       ??_C@_0CB@PJFPAIKJ@JVMTI_ERROR_INVALID_THREAD_GROU@ 00000001800059d8     libsetlocal001.obj
 0002:00000a00       ??_C@_0BN@LLMKHMNF@JVMTI_ERROR_INVALID_PRIORITY@ 0000000180005a00     libsetlocal001.obj
 0002:00000a20       ??_C@_0CB@MBOFKAGB@JVMTI_ERROR_THREAD_NOT_SUSPENDE@ 0000000180005a20     libsetlocal001.obj
 0002:00000a48       ??_C@_0BN@FABOLPBI@JVMTI_ERROR_THREAD_SUSPENDED@ 0000000180005a48     libsetlocal001.obj
 0002:00000a68       ??_C@_0BN@FDGNOBJM@JVMTI_ERROR_THREAD_NOT_ALIVE@ 0000000180005a68     libsetlocal001.obj
 0002:00000a88       ??_C@_0BL@GOBIFKNJ@JVMTI_ERROR_INVALID_OBJECT@ 0000000180005a88     libsetlocal001.obj
 0002:00000aa8       ??_C@_0BK@FCMAJPPC@JVMTI_ERROR_INVALID_CLASS@ 0000000180005aa8     libsetlocal001.obj
 0002:00000ac8       ??_C@_0BP@IKLLBKEB@JVMTI_ERROR_CLASS_NOT_PREPARED@ 0000000180005ac8     libsetlocal001.obj
 0002:00000ae8       ??_C@_0BN@KLPPLKG@JVMTI_ERROR_INVALID_METHODID@ 0000000180005ae8     libsetlocal001.obj
 0002:00000b08       ??_C@_0BN@BCEKOKND@JVMTI_ERROR_INVALID_LOCATION@ 0000000180005b08     libsetlocal001.obj
 0002:00000b28       ??_C@_0BM@DFDGPME@JVMTI_ERROR_INVALID_FIELDID@ 0000000180005b28     libsetlocal001.obj
 0002:00000b48       ??_C@_0BL@NELIEPEC@JVMTI_ERROR_NO_MORE_FRAMES@ 0000000180005b48     libsetlocal001.obj
 0002:00000b68       ??_C@_0BJ@BDBECFDM@JVMTI_ERROR_OPAQUE_FRAME@ 0000000180005b68     libsetlocal001.obj
 0002:00000b88       ??_C@_0BK@MIIFNLOB@JVMTI_ERROR_TYPE_MISMATCH@ 0000000180005b88     libsetlocal001.obj
 0002:00000ba8       ??_C@_0BJ@HPCAOILC@JVMTI_ERROR_INVALID_SLOT@ 0000000180005ba8     libsetlocal001.obj
 0002:00000bc8       ??_C@_0BG@CHILOPNI@JVMTI_ERROR_DUPLICATE@ 0000000180005bc8     libsetlocal001.obj
 0002:00000be0       ??_C@_0BG@DIEMLHKM@JVMTI_ERROR_NOT_FOUND@ 0000000180005be0     libsetlocal001.obj
 0002:00000bf8       ??_C@_0BM@NHMCKHOB@JVMTI_ERROR_INVALID_MONITOR@ 0000000180005bf8     libsetlocal001.obj
 0002:00000c18       ??_C@_0BO@PPEDAJGL@JVMTI_ERROR_NOT_MONITOR_OWNER@ 0000000180005c18     libsetlocal001.obj
 0002:00000c38       ??_C@_0BG@FCAIPEID@JVMTI_ERROR_INTERRUPT@ 0000000180005c38     libsetlocal001.obj
 0002:00000c50       ??_C@_0CB@EGDBNKOI@JVMTI_ERROR_INVALID_CLASS_FORMA@ 0000000180005c50     libsetlocal001.obj
 0002:00000c78       ??_C@_0CG@DGKOGIAL@JVMTI_ERROR_CIRCULAR_CLASS_DEFI@ 0000000180005c78     libsetlocal001.obj
 0002:00000ca0       ??_C@_0BP@ICEALPKC@JVMTI_ERROR_FAILS_VERIFICATION@ 0000000180005ca0     libsetlocal001.obj
 0002:00000cc0       ??_C@_0DC@JDACLMIO@JVMTI_ERROR_UNSUPPORTED_REDEFIN@ 0000000180005cc0     libsetlocal001.obj
 0002:00000cf8       ??_C@_0DE@GKDKNOMJ@JVMTI_ERROR_UNSUPPORTED_REDEFIN@ 0000000180005cf8     libsetlocal001.obj
 0002:00000d30       ??_C@_0BO@LAFKIOG@JVMTI_ERROR_INVALID_TYPESTATE@ 0000000180005d30     libsetlocal001.obj
 0002:00000d50       ??_C@_0DH@INDGCLLB@JVMTI_ERROR_UNSUPPORTED_REDEFIN@ 0000000180005d50     libsetlocal001.obj
 0002:00000d88       ??_C@_0DE@NHEOMMGI@JVMTI_ERROR_UNSUPPORTED_REDEFIN@ 0000000180005d88     libsetlocal001.obj
 0002:00000dc0       ??_C@_0CA@EKPNJOEP@JVMTI_ERROR_UNSUPPORTED_VERSION@ 0000000180005dc0     libsetlocal001.obj
 0002:00000de0       ??_C@_0BN@OFFMAHHL@JVMTI_ERROR_NAMES_DONT_MATCH@ 0000000180005de0     libsetlocal001.obj
 0002:00000e00       ??_C@_0DN@HHBBLAKE@JVMTI_ERROR_UNSUPPORTED_REDEFIN@ 0000000180005e00     libsetlocal001.obj
 0002:00000e40       ??_C@_0DO@HMBGBGNA@JVMTI_ERROR_UNSUPPORTED_REDEFIN@ 0000000180005e40     libsetlocal001.obj
 0002:00000e80       ??_C@_0BP@PBECGKHJ@JVMTI_ERROR_UNMODIFIABLE_CLASS@ 0000000180005e80     libsetlocal001.obj
 0002:00000ea0       ??_C@_0BK@CANILEHF@JVMTI_ERROR_NOT_AVAILABLE@ 0000000180005ea0     libsetlocal001.obj
 0002:00000ec0       ??_C@_0CE@INJKMEFK@JVMTI_ERROR_MUST_POSSESS_CAPABI@ 0000000180005ec0     libsetlocal001.obj
 0002:00000ee8       ??_C@_0BJ@LBFPFPDM@JVMTI_ERROR_NULL_POINTER@ 0000000180005ee8     libsetlocal001.obj
 0002:00000f08       ??_C@_0BP@CHJPNNEM@JVMTI_ERROR_ABSENT_INFORMATION@ 0000000180005f08     libsetlocal001.obj
 0002:00000f28       ??_C@_0BP@OMFMNLC@JVMTI_ERROR_INVALID_EVENT_TYPE@ 0000000180005f28     libsetlocal001.obj
 0002:00000f48       ??_C@_0BN@BIBNPHHO@JVMTI_ERROR_ILLEGAL_ARGUMENT@ 0000000180005f48     libsetlocal001.obj
 0002:00000f68       ??_C@_0BK@KKNDHDCE@JVMTI_ERROR_NATIVE_METHOD@ 0000000180005f68     libsetlocal001.obj
 0002:00000f88       ??_C@_0BK@PMKCFHAE@JVMTI_ERROR_OUT_OF_MEMORY@ 0000000180005f88     libsetlocal001.obj
 0002:00000fa8       ??_C@_0BK@NNJBDMNB@JVMTI_ERROR_ACCESS_DENIED@ 0000000180005fa8     libsetlocal001.obj
 0002:00000fc8       ??_C@_0BI@GHECLMNC@JVMTI_ERROR_WRONG_PHASE@ 0000000180005fc8     libsetlocal001.obj
 0002:00000fe0       ??_C@_0BF@OLIHJOII@JVMTI_ERROR_INTERNAL@ 0000000180005fe0     libsetlocal001.obj
 0002:00000ff8       ??_C@_0BO@EOHGKJHI@JVMTI_ERROR_UNATTACHED_THREAD@ 0000000180005ff8     libsetlocal001.obj
 0002:00001018       ??_C@_0CA@LKHFDACL@JVMTI_ERROR_INVALID_ENVIRONMENT@ 0000000180006018     libsetlocal001.obj
 0002:00001038       ??_C@_0BA@MMFHLOKK@?$DMunknown?5error?$DO@ 0000000180006038     libsetlocal001.obj
 0002:00001048       ??_C@_0CF@CBHOKDB@throwable?5?$DN?5jni?9?$DOExceptionOccur@ 0000000180006048     libsetlocal001.obj
 0002:00001070       ??_C@_03OFAPEBGM@?$CFs?6@  0000000180006070     libsetlocal001.obj
 0002:00001078       ??_C@_0DM@LPIGEGNJ@s?2test?2hotspot?2jtreg?2vmTestbase@ 0000000180006078     libsetlocal001.obj
 0002:000010b8       ??_C@_0CC@NFCNPEPK@Exception?5in?5JNI?5call?5?$CIcleared?$CJ@ 00000001800060b8     libsetlocal001.obj
 0002:000010e0       ??_C@_0BJ@IBAKFIKF@jni?9?$DOExceptionDescribe?$CI?$CJ@ 00000001800060e0     libsetlocal001.obj
 0002:00001100       ??_C@_0BG@GGKALKMH@jni?9?$DOExceptionClear?$CI?$CJ@ 0000000180006100     libsetlocal001.obj
 0002:00001118       ??_C@_0CF@JMGFGJLJ@?$CD?5?5?5verified?5JNI?5assertion?5is?5F@ 0000000180006118     libsetlocal001.obj
 0002:00001140       ??_C@_0CB@MLNJNCLJ@?5?5jvmti?5error?3?5code?$DN?$CFd?0?5name?$DN?$CFs@ 0000000180006140     libsetlocal001.obj
 0002:00001168       ??_C@_0CD@OHBGDKMK@?$CD?5?5?5jvmti?5error?3?5code?$DN?$CFd?0?5name?$DN@ 0000000180006168     libsetlocal001.obj
 0002:00001190       ??_C@_0CG@JNNCGPHB@?$CD?5?5?5error?5expected?3?5code?$DN?$CFd?0?5na@ 0000000180006190     libsetlocal001.obj
 0002:000011c0       ??_C@_0EB@IMGKPCGE@?$CIstr_obj?5?$DN?5jni?9?$DONewStringUTF?$CIco@ 00000001800061c0     libsetlocal001.obj
 0002:00001210       ??_C@_0EA@HFOGGBCC@s?2test?2hotspot?2jtreg?2vmTestbase@ 0000000180006210     libsetlocal001.obj
 0002:00001250       ??_C@_0CO@HJKAMPK@?$CIGetFrameLocation?$CJ?5unexpected?5e@ 0000000180006250     libsetlocal001.obj
 0002:00001280       ??_C@_05KKCIMGE@error@     0000000180006280     libsetlocal001.obj
 0002:00001288       ??_C@_0CJ@JACLEAA@Test?5failed?5by?5setFailStatus?$CI?$CJ?4@ 0000000180006288     libsetlocal001.obj
 0002:000012c0       ??_C@_0EA@PNBCDMOA@s?2test?2hotspot?2jtreg?2vmTestbase@ 00000001800062c0     libsetlocal001.obj
 0002:00001300       ??_C@_0DI@ILAHDLMP@?$CI?$CKagentThreadProc?$CJ?$CIjvmti_env?0?5a@ 0000000180006300     libsetlocal001.obj
 0002:00001338       ??_C@_0BD@KDBALNLB@JVMTI?5agent?5thread@ 0000000180006338     libsetlocal001.obj
 0002:00001350       ??_C@_0BB@NOKBFPFO@java?1lang?1Thread@ 0000000180006350     libsetlocal001.obj
 0002:00001364       ??_C@_06FALKBLGB@?$DMinit?$DO@ 0000000180006364     libsetlocal001.obj
 0002:00001370       ??_C@_0BG@IKDDPPGD@?$CILjava?1lang?1String?$DL?$CJV@ 0000000180006370     libsetlocal001.obj
 0002:00001390       ??_C@_0EB@IFJBFEKC@?$CIthreadClass?5?$DN?5jni_env?9?$DOFindCla@ 0000000180006390     libsetlocal001.obj
 0002:000013e0       ??_C@_0GF@FGFIBKKL@?$CIthreadCtor?5?$DN?5jni_env?9?$DOGetMetho@ 00000001800063e0     libsetlocal001.obj
 0002:00001448       ??_C@_0DN@NCPDJLOG@?$CIthreadName?5?$DN?5jni_env?9?$DONewStrin@ 0000000180006448     libsetlocal001.obj
 0002:00001490       ??_C@_0FE@PFKODBGC@?$CIthreadObject?5?$DN?5jni_env?9?$DONewObj@ 0000000180006490     libsetlocal001.obj
 0002:000014f0       ??_C@_0ED@HOBAHHJI@?$CIthreadGlobalRef?5?$DN?5jni_env?9?$DONew@ 00000001800064f0     libsetlocal001.obj
 0002:00001540       ??_C@_0FN@HNJJAHFC@jvmti_env?9?$DORunAgentThread?$CIagent@ 0000000180006540     libsetlocal001.obj
 0002:000015a0       ??_C@_0EA@MOJDNKDF@Debuggee?5status?5sync?5aborted?5be@ 00000001800065a0     libsetlocal001.obj
 0002:000015e0       ??_C@_0EA@EEOEJAEN@status?5?$DN?5syncDebuggeeStatus?$CIjni@ 00000001800065e0     libsetlocal001.obj
 0002:00001620       ??_C@_0BL@JBCFNBMB@nsk_jvmti_resetAgentData?$CI?$CJ@ 0000000180006620     libsetlocal001.obj
 0002:00001640       ??_C@_0EL@LPBEELIP@s?2test?2hotspot?2jtreg?2vmTestbase@ 0000000180006640     libsetlocal001.obj
 0002:00001690       ??_C@_0CK@JDAMFDMJ@jvmti?9?$DOSetTag?$CIo?0?5tag?$CJ?5?$DN?$DN?5JVMTI_@ 0000000180006690     libsetlocal001.obj
 0002:000016c0       ??_C@_0CC@DAMNHKNI@Can?8t?5set?5tag?5?$CFli?5for?5object?5?$CFl@ 00000001800066c0     libsetlocal001.obj
 0002:000016e8       ??_C@_0DL@HAJPNKEF@jvmti?9?$DOGetObjectHashCode?$CIo?0?5?$CGha@ 00000001800066e8     libsetlocal001.obj
 0002:00001728       ??_C@_0BL@JFPIEOBF@Can?8t?5get?5hash?5object?5?$CFlx?6@ 0000000180006728     libsetlocal001.obj
 0002:00001748       ??_C@_0BG@DICPHBKN@setTag?3?5?$CF08x?5?$DM?9?5?$CF?53li@ 0000000180006748     libsetlocal001.obj
 0002:00001760       ??_C@_0DH@FCEEBDMJ@?$CIs?5?$DN?5jni?9?$DOGetStringUTFChars?$CIsIn@ 0000000180006760     libsetlocal001.obj
 0002:00001798       ??_C@_0BJ@OKKGHDCN@Can?8t?5get?5string?5at?5?$CF?$CDp?6@ 0000000180006798     libsetlocal001.obj
 0002:000017b8       ??_C@_0BP@EKFLGGFJ@Can?8t?5get?5string?5at?5?$CF?$CDp?3?5null?6@ 00000001800067b8     libsetlocal001.obj
 0002:000017d8       ??_C@_06ICODBHCL@?5?1?1?5?$CFs@ 00000001800067d8     libsetlocal001.obj
 0002:000017e0       ??_C@_0DB@KGFPLEGO@?$CIr?5?$DN?5jvmti?9?$DOGetTag?$CIo?0?5?$CGtag?$CJ?$CJ?5?$DN?$DN@ 00000001800067e0     libsetlocal001.obj
 0002:00001818       ??_C@_0CO@PDAGBCGJ@Can?8t?5GetTag?5for?5object?5?$CFlx?4?5Re@ 0000000180006818     libsetlocal001.obj
 0002:00001848       ??_C@_0CH@HPEODOHC@TEST_BUG?3?5Max?4?5number?5of?5refs?5r@ 0000000180006848     libsetlocal001.obj
 0002:00001870       ??_C@_0DI@PHFCABIM@?$CIr?5?$DN?5jvmti?9?$DOGetTag?$CIfrom?0?5?$CGtagFr@ 0000000180006870     libsetlocal001.obj
 0002:000018a8       ??_C@_0DI@MDEGFNKD@TEST_BUG?3?5Can?8t?5GetTag?5for?5obje@ 00000001800068a8     libsetlocal001.obj
 0002:000018e0       ??_C@_0DE@MLELJAHM@?$CIr?5?$DN?5jvmti?9?$DOGetTag?$CIto?0?5?$CGtagTo?$CJ?$CJ@ 00000001800068e0     libsetlocal001.obj
 0002:00001914       ??_C@_03GAEACAIP@?$CI?$CJV@ 0000000180006914     libsetlocal001.obj
 0002:00001918       ??_C@_0CA@JOLKCKMH@?$CI?$CFs?$CJ?5unexpected?5error?3?5?$CFs?5?$CI?$CFd?$CJ?6@ 0000000180006918     libsetlocal001.obj
 0002:00001938       ??_C@_0DD@ELHIJBGO@?$CIGetLocalVariableTable?$CJ?5unexpec@ 0000000180006938     libsetlocal001.obj
 0002:0000196c       ??_C@_01HHGOMJKL@l@        000000018000696c     libsetlocal001.obj
 0002:00001970       ??_C@_0N@CHLNBHIP@SetLocalLong@ 0000000180006970     libsetlocal001.obj
 0002:00001980       ??_C@_01INIBCBCB@f@        0000000180006980     libsetlocal001.obj
 0002:00001988       ??_C@_0O@GMHJNNDF@SetLocalFloat@ 0000000180006988     libsetlocal001.obj
 0002:00001998       ??_C@_01LPLHEDKD@d@        0000000180006998     libsetlocal001.obj
 0002:000019a0       ??_C@_0P@HFIOJDJO@SetLocalDouble@ 00000001800069a0     libsetlocal001.obj
 0002:000019b0       ??_C@_02IBOFNBPA@i1@       00000001800069b0     libsetlocal001.obj
 0002:000019b8       ??_C@_0P@BJNBGNKI@SetLocalInt?$CDi1@ 00000001800069b8     libsetlocal001.obj
 0002:000019c8       ??_C@_02KKMIICDD@i2@       00000001800069c8     libsetlocal001.obj
 0002:000019d0       ??_C@_0P@DCPMDOGL@SetLocalInt?$CDi2@ 00000001800069d0     libsetlocal001.obj
 0002:000019e0       ??_C@_02LDNDLDHC@i3@       00000001800069e0     libsetlocal001.obj
 0002:000019e8       ??_C@_0P@CLOHAPCK@SetLocalInt?$CDi3@ 00000001800069e8     libsetlocal001.obj
 0002:000019f8       ??_C@_02PMJCCFLF@i4@       00000001800069f8     libsetlocal001.obj
 0002:00001a00       ??_C@_0P@GEKGJJON@SetLocalInt?$CDi4@ 0000000180006a00     libsetlocal001.obj
 0002:00001a10       ??_C@_02OFIJBEPE@i5@       0000000180006a10     libsetlocal001.obj
 0002:00001a18       ??_C@_0P@HNLNKIKM@SetLocalInt?$CDi5@ 0000000180006a18     libsetlocal001.obj
 0002:00001a28       ??_C@_03DAPANPEK@ob1@      0000000180006a28     libsetlocal001.obj
 0002:00001a30       ??_C@_0BD@NOCOCDKP@SetLocalObject?$CDob1@ 0000000180006a30     libsetlocal001.obj
 0002:00001a44       ??_C@_03BLNNIMIJ@ob2@      0000000180006a44     libsetlocal001.obj
 0002:00001a48       ??_C@_0BD@PFADHAGM@SetLocalObject?$CDob2@ 0000000180006a48     libsetlocal001.obj
 0002:00001a60       ??_C@_0BF@OGOPLKEC@SetLocalInt?$CDi1?0param@ 0000000180006a60     libsetlocal001.obj
 0002:00001a78       ??_C@_0BF@GIGALNKB@SetLocalInt?$CDi2?0param@ 0000000180006a78     libsetlocal001.obj
 0002:00001a90       ??_C@_0BF@KEMKLNDP@SetLocalInt?$CDi3?0param@ 0000000180006a90     libsetlocal001.obj
 0002:00001aa8       ??_C@_0BF@KOAPLECG@SetLocalInt?$CDi4?0param@ 0000000180006aa8     libsetlocal001.obj
 0002:00001ac0       ??_C@_01OJONOECF@b@        0000000180006ac0     libsetlocal001.obj
 0002:00001ac8       ??_C@_0BE@DCDDGDBI@SetLocalInt?$CDb?0param@ 0000000180006ac8     libsetlocal001.obj
 0002:00001ae0       ??_C@_0BD@BACBPHID@SetLocalLong?0param@ 0000000180006ae0     libsetlocal001.obj
 0002:00001af8       ??_C@_0BE@INDFCMJK@SetLocalFloat?0param@ 0000000180006af8     libsetlocal001.obj
 0002:00001b10       ??_C@_0BF@BBGLJNHO@SetLocalDouble?0param@ 0000000180006b10     libsetlocal001.obj
 0002:00001b28       ??_C@_0CM@EGMIFBJC@ERROR?3?5didn?8t?5know?5where?5we?5got@ 0000000180006b28     libsetlocal001.obj
 0002:00001b58       ??_C@_0CK@DEFLIKCM@Wrong?5result?5of?5a?5valid?5call?5to@ 0000000180006b58     libsetlocal001.obj
 0002:00001b88       ??_C@_0DG@LAJPGIIE@?$CIGetPotentialCapabilities?$CJ?5unex@ 0000000180006b88     libsetlocal001.obj
 0002:00001bc0       ??_C@_0CN@LKPEOJPO@?$CIAddCapabilities?$CJ?5unexpected?5er@ 0000000180006bc0     libsetlocal001.obj
 0002:00001bf0       ??_C@_0CN@BCCBOHCH@?$CIGetCapabilities?$CJ?5unexpected?5er@ 0000000180006bf0     libsetlocal001.obj
 0002:00001c20       ??_C@_0DH@IJEIPLEC@Warning?3?5access?5to?5local?5variab@ 0000000180006c20     libsetlocal001.obj
 0002:00001c58       ??_C@_0CP@IMINGNLL@?$CISetEventCallbacks?$CJ?5unexpected?5@ 0000000180006c58     libsetlocal001.obj
 0002:00001c88       ??_C@_0CO@FDBBPEKA@Warning?3?5Breakpoint?5event?5is?5no@ 0000000180006c88     libsetlocal001.obj
 0002:00001cb8       ??_C@_0CH@CDOJMNAO@JVMTI?5client?5was?5not?5properly?5l@ 0000000180006cb8     libsetlocal001.obj
 0002:00001ce0       ??_C@_0L@GIHILDI@checkPoint@ 0000000180006ce0     libsetlocal001.obj
 0002:00001cec       ??_C@_03BILEFAFM@?$CI?$CJD@ 0000000180006cec     libsetlocal001.obj
 0002:00001cf0       ??_C@_06MADNOIIM@meth01@   0000000180006cf0     libsetlocal001.obj
 0002:00001cf8       ??_C@_04PFANPMCN@?$CII?$CJV@ 0000000180006cf8     libsetlocal001.obj
 0002:00001d00       ??_C@_06OLBALLEP@meth02@   0000000180006d00     libsetlocal001.obj
 0002:00001d08       ??_C@_06PCALIKAO@meth03@   0000000180006d08     libsetlocal001.obj
 0002:00001d10       ??_C@_0M@KJJOHAPG@?$CIIJSDCFBZ?$CJV@ 0000000180006d10     libsetlocal001.obj
 0002:00001d1c       ??_C@_06LNEKBMMJ@meth04@   0000000180006d1c     libsetlocal001.obj
 0002:00001d28       ??_C@_0CE@HCBNHAFL@Cannot?5find?5Method?5ID?5for?5a?5met@ 0000000180006d28     libsetlocal001.obj
 0002:00001d50       ??_C@_0CC@GAODDEMK@Failed?5to?5SetBreakpoint?3?5?$CFs?5?$CI?$CFd@ 0000000180006d50     libsetlocal001.obj
 0002:00001d78       ??_C@_0CM@NEGFNKGE@Failed?5to?5enable?5BREAKPOINT?5eve@ 0000000180006d78     libsetlocal001.obj
 0002:00001dc0       ??_C@_1EC@JIJBPKFM@?$AAa?$AAp?$AAi?$AA?9?$AAm?$AAs?$AA?9?$AAw?$AAi?$AAn?$AA?9?$AAc?$AAo?$AAr?$AAe@ 0000000180006dc0     MSVCRT:thread_safe_statics.obj
 0002:00001e08       ??_C@_1BK@MGMFAEKH@?$AAk?$AAe?$AAr?$AAn?$AAe?$AAl?$AA3?$AA2?$AA?4?$AAd?$AAl?$AAl@ 0000000180006e08     MSVCRT:thread_safe_statics.obj
 0002:00001e28       ??_C@_0BJ@JEBJOJFJ@SleepConditionVariableCS@ 0000000180006e28     MSVCRT:thread_safe_statics.obj
 0002:00001e48       ??_C@_0BJ@PGPPEPCC@WakeAllConditionVariable@ 0000000180006e48     MSVCRT:thread_safe_statics.obj
 0002:00001e68       _pDefaultRawDllMain        0000000180006e68     MSVCRT:dll_dllmain.obj
 0002:00001e68       _pRawDllMain               0000000180006e68     MSVCRT:dll_dllmain.obj
 0002:00001e70       __xmm@ffffffffffffffffffffffffffffffff 0000000180006e70     MSVCRT:utility.obj
 0002:00001e80       _load_config_used          0000000180006e80     MSVCRT:loadcfg.obj
 0002:00002080       _tls_used                  0000000180007080     MSVCRT:tlssup.obj
 0002:000020a8       __volatile_metadata        00000001800070a8     <linker-defined>
 0002:00002468       __rtc_iaa                  0000000180007468     MSVCRT:initsect.obj
 0002:00002470       __rtc_izz                  0000000180007470     MSVCRT:initsect.obj
 0002:00002478       __rtc_taa                  0000000180007478     MSVCRT:initsect.obj
 0002:00002480       __rtc_tzz                  0000000180007480     MSVCRT:initsect.obj
 0002:00002488       _tls_start                 0000000180007488     MSVCRT:tlssup.obj
 0002:0000248c       _Init_thread_epoch         000000018000748c     MSVCRT:thread_safe_statics.obj
 0002:00002490       _tls_end                   0000000180007490     MSVCRT:tlssup.obj
 0002:00002b94       __IMPORT_DESCRIPTOR_KERNEL32 0000000180007b94     kernel32:KERNEL32.dll
 0002:00002ba8       __IMPORT_DESCRIPTOR_VCRUNTIME140 0000000180007ba8     vcruntime:VCRUNTIME140.dll
 0002:00002bbc       __IMPORT_DESCRIPTOR_api-ms-win-crt-runtime-l1-1-0 0000000180007bbc     ucrt:api-ms-win-crt-runtime-l1-1-0.dll
 0002:00002bd0       __IMPORT_DESCRIPTOR_api-ms-win-crt-stdio-l1-1-0 0000000180007bd0     ucrt:api-ms-win-crt-stdio-l1-1-0.dll
 0002:00002be4       __IMPORT_DESCRIPTOR_api-ms-win-crt-string-l1-1-0 0000000180007be4     ucrt:api-ms-win-crt-string-l1-1-0.dll
 0002:00002bf8       __NULL_IMPORT_DESCRIPTOR   0000000180007bf8     kernel32:KERNEL32.dll
 0003:00000038       _Init_global_epoch         0000000180009038     MSVCRT:thread_safe_statics.obj
 0003:00000040       __security_cookie          0000000180009040     MSVCRT:gs_cookie.obj
 0003:00000048       __security_cookie_complement 0000000180009048     MSVCRT:gs_cookie.obj
 0003:00000050       _fltused                   0000000180009050     MSVCRT:fltused.obj
 0003:00000054       __scrt_native_dllmain_reason 0000000180009054     MSVCRT:utility.obj
 0003:00000058       __isa_available            0000000180009058     MSVCRT:cpu_disp.obj
 0003:0000005c       __isa_enabled              000000018000905c     MSVCRT:cpu_disp.obj
 0003:00000060       __memset_fast_string_threshold 0000000180009060     MSVCRT:cpu_disp.obj
 0003:00000068       __memset_nt_threshold      0000000180009068     MSVCRT:cpu_disp.obj
 0003:00000070       __scrt_ucrt_dll_is_in_use  0000000180009070     MSVCRT:ucrt_stubs.obj
 0003:00000080       g_wrongHeapCallbacks       0000000180009080     libsetlocal001.obj
 0003:00000100       g_szTagInfo                0000000180009100     libsetlocal001.obj
 0003:00002040       g_tagFlags                 000000018000b040     libsetlocal001.obj
 0003:00002428       g_refsToVerifyCnt          000000018000b428     libsetlocal001.obj
 0003:0000242c       g_fakeUserData             000000018000b42c     libsetlocal001.obj
 0003:00002430       g_tagVisitCount            000000018000b430     libsetlocal001.obj
 0003:000033d0       g_refsToVerify             000000018000c3d0     libsetlocal001.obj
 0003:0001aad0       g_userDataError            0000000180023ad0     libsetlocal001.obj
 0003:0001adf8       ?_OptionsStorage@?1??__local_stdio_printf_options@@9@4_KA 0000000180023df8     libsetlocal001.obj
 0003:0001b3b8       _tls_index                 00000001800243b8     MSVCRT:tlssup.obj
 0003:0001b3c0       __scrt_current_native_startup_state 00000001800243c0     MSVCRT:utility.obj
 0003:0001b3c8       __scrt_native_startup_lock 00000001800243c8     MSVCRT:utility.obj
 0003:0001b408       __scrt_debugger_hook_flag  0000000180024408     MSVCRT:utility_desktop.obj
 0003:0001b410       ?__type_info_root_node@@3U__type_info_node@@A 0000000180024410     MSVCRT:tncleanup.obj
 0003:0001b420       ?_OptionsStorage@?1??__local_stdio_scanf_options@@9@4_KA 0000000180024420     MSVCRT:default_local_stdio_options.obj
 0003:0001b428       __favor                    0000000180024428     MSVCRT:cpu_disp.obj
 0003:0001b430       __dyn_tls_init_callback    0000000180024430     <common>

 entry point at        0001:00002bd0

 Static symbols

 0000:fffd9000       .debug$S                   0000000180000000     setlocal001.exp
 0000:fffd9000       .debug$S                   0000000180000000     vcruntime:VCRUNTIME140.dll
 0000:fffd9000       .debug$S                   0000000180000000     vcruntime:VCRUNTIME140.dll
 0000:fffd9000       .debug$S                   0000000180000000     vcruntime:VCRUNTIME140.dll
 0000:fffd9000       .debug$S                   0000000180000000     vcruntime:VCRUNTIME140.dll
 0000:fffd9000       .debug$S                   0000000180000000     vcruntime:VCRUNTIME140.dll
 0000:fffd9000       .debug$S                   0000000180000000     vcruntime:VCRUNTIME140.dll
 0000:fffd9000       .debug$S                   0000000180000000     vcruntime:VCRUNTIME140.dll
 0000:fffd9000       .debug$S                   0000000180000000     ucrt:api-ms-win-crt-convert-l1-1-0.dll
 0002:ffffb000       .idata$6                   0000000180000000     ucrt:api-ms-win-crt-convert-l1-1-0.dll
 0000:fffd9000       .debug$S                   0000000180000000     ucrt:api-ms-win-crt-heap-l1-1-0.dll
 0000:fffd9000       .debug$S                   0000000180000000     ucrt:api-ms-win-crt-heap-l1-1-0.dll
 0000:fffd9000       .debug$S                   0000000180000000     ucrt:api-ms-win-crt-heap-l1-1-0.dll
 0000:fffd9000       .debug$S                   0000000180000000     ucrt:api-ms-win-crt-heap-l1-1-0.dll
 0002:ffffb000       .idata$6                   0000000180000000     ucrt:api-ms-win-crt-heap-l1-1-0.dll
 0000:fffd9000       .debug$S                   0000000180000000     ucrt:api-ms-win-crt-runtime-l1-1-0.dll
 0000:fffd9000       .debug$S                   0000000180000000     ucrt:api-ms-win-crt-runtime-l1-1-0.dll
 0000:fffd9000       .debug$S                   0000000180000000     ucrt:api-ms-win-crt-runtime-l1-1-0.dll
 0000:fffd9000       .debug$S                   0000000180000000     ucrt:api-ms-win-crt-runtime-l1-1-0.dll
 0000:fffd9000       .debug$S                   0000000180000000     ucrt:api-ms-win-crt-runtime-l1-1-0.dll
 0000:fffd9000       .debug$S                   0000000180000000     ucrt:api-ms-win-crt-runtime-l1-1-0.dll
 0000:fffd9000       .debug$S                   0000000180000000     ucrt:api-ms-win-crt-runtime-l1-1-0.dll
 0000:fffd9000       .debug$S                   0000000180000000     ucrt:api-ms-win-crt-runtime-l1-1-0.dll
 0000:fffd9000       .debug$S                   0000000180000000     ucrt:api-ms-win-crt-runtime-l1-1-0.dll
 0000:fffd9000       .debug$S                   0000000180000000     ucrt:api-ms-win-crt-runtime-l1-1-0.dll
 0000:fffd9000       .debug$S                   0000000180000000     ucrt:api-ms-win-crt-runtime-l1-1-0.dll
 0000:fffd9000       .debug$S                   0000000180000000     ucrt:api-ms-win-crt-runtime-l1-1-0.dll
 0000:fffd9000       .debug$S                   0000000180000000     ucrt:api-ms-win-crt-runtime-l1-1-0.dll
 0000:fffd9000       .debug$S                   0000000180000000     ucrt:api-ms-win-crt-runtime-l1-1-0.dll
 0000:fffd9000       .debug$S                   0000000180000000     ucrt:api-ms-win-crt-runtime-l1-1-0.dll
 0000:fffd9000       .debug$S                   0000000180000000     ucrt:api-ms-win-crt-runtime-l1-1-0.dll
 0000:fffd9000       .debug$S                   0000000180000000     ucrt:api-ms-win-crt-stdio-l1-1-0.dll
 0000:fffd9000       .debug$S                   0000000180000000     ucrt:api-ms-win-crt-stdio-l1-1-0.dll
 0000:fffd9000       .debug$S                   0000000180000000     ucrt:api-ms-win-crt-stdio-l1-1-0.dll
 0000:fffd9000       .debug$S                   0000000180000000     ucrt:api-ms-win-crt-stdio-l1-1-0.dll
 0000:fffd9000       .debug$S                   0000000180000000     ucrt:api-ms-win-crt-stdio-l1-1-0.dll
 0000:fffd9000       .debug$S                   0000000180000000     ucrt:api-ms-win-crt-stdio-l1-1-0.dll
 0000:fffd9000       .debug$S                   0000000180000000     ucrt:api-ms-win-crt-stdio-l1-1-0.dll
 0000:fffd9000       .debug$S                   0000000180000000     ucrt:api-ms-win-crt-stdio-l1-1-0.dll
 0000:fffd9000       .debug$S                   0000000180000000     ucrt:api-ms-win-crt-stdio-l1-1-0.dll
 0000:fffd9000       .debug$S                   0000000180000000     ucrt:api-ms-win-crt-stdio-l1-1-0.dll
 0000:fffd9000       .debug$S                   0000000180000000     ucrt:api-ms-win-crt-string-l1-1-0.dll
 0000:fffd9000       .debug$S                   0000000180000000     ucrt:api-ms-win-crt-string-l1-1-0.dll
 0000:fffd9000       .debug$S                   0000000180000000     ucrt:api-ms-win-crt-string-l1-1-0.dll
 0000:fffd9000       .debug$S                   0000000180000000     ucrt:api-ms-win-crt-string-l1-1-0.dll
 0000:fffd9000       .debug$S                   0000000180000000     ucrt:api-ms-win-crt-string-l1-1-0.dll
 0000:fffd9000       .debug$S                   0000000180000000     ucrt:api-ms-win-crt-string-l1-1-0.dll
 0000:fffd9000       .debug$S                   0000000180000000     ucrt:api-ms-win-crt-string-l1-1-0.dll
 0000:fffd9000       .debug$S                   0000000180000000     ucrt:api-ms-win-crt-string-l1-1-0.dll
 0000:fffd9000       .debug$S                   0000000180000000     kernel32:KERNEL32.dll
 0000:fffd9000       .debug$S                   0000000180000000     kernel32:KERNEL32.dll
 0000:fffd9000       .debug$S                   0000000180000000     kernel32:KERNEL32.dll
 0000:fffd9000       .debug$S                   0000000180000000     kernel32:KERNEL32.dll
 0000:fffd9000       .debug$S                   0000000180000000     kernel32:KERNEL32.dll
 0000:fffd9000       .debug$S                   0000000180000000     kernel32:KERNEL32.dll
 0000:fffd9000       .debug$S                   0000000180000000     kernel32:KERNEL32.dll
 0000:fffd9000       .debug$S                   0000000180000000     kernel32:KERNEL32.dll
 0000:fffd9000       .debug$S                   0000000180000000     kernel32:KERNEL32.dll
 0000:fffd9000       .debug$S                   0000000180000000     kernel32:KERNEL32.dll
 0000:fffd9000       .debug$S                   0000000180000000     kernel32:KERNEL32.dll
 0000:fffd9000       .debug$S                   0000000180000000     kernel32:KERNEL32.dll
 0000:fffd9000       .debug$S                   0000000180000000     kernel32:KERNEL32.dll
 0000:fffd9000       .debug$S                   0000000180000000     kernel32:KERNEL32.dll
 0000:fffd9000       .debug$S                   0000000180000000     kernel32:KERNEL32.dll
 0000:fffd9000       .debug$S                   0000000180000000     kernel32:KERNEL32.dll
 0000:fffd9000       .debug$S                   0000000180000000     kernel32:KERNEL32.dll
 0000:fffd9000       .debug$S                   0000000180000000     kernel32:KERNEL32.dll
 0000:fffd9000       .debug$S                   0000000180000000     kernel32:KERNEL32.dll
 0000:fffd9000       .debug$S                   0000000180000000     kernel32:KERNEL32.dll
 0000:fffd9000       .debug$S                   0000000180000000     kernel32:KERNEL32.dll
 0000:fffd9000       .debug$S                   0000000180000000     kernel32:KERNEL32.dll
 0000:fffd9000       .debug$S                   0000000180000000     kernel32:KERNEL32.dll
 0000:fffd9000       .debug$S                   0000000180000000     kernel32:KERNEL32.dll
 0000:fffd9000       .debug$S                   0000000180000000     kernel32:KERNEL32.dll
 0000:fffd9000       .debug$S                   0000000180000000     kernel32:KERNEL32.dll
 0000:fffd9000       .debug$S                   0000000180000000     kernel32:KERNEL32.dll
 0000:fffd9000       .debug$S                   0000000180000000     kernel32:KERNEL32.dll
 0001:000017a0       addRefToVerify             00000001800027a0 f   libsetlocal001.obj
 0001:0000180c       agentThreadWrapper         000000018000280c f   libsetlocal001.obj
 0001:00001978       check_error                0000000180002978 f   libsetlocal001.obj
 0001:00001a48       file_basename              0000000180002a48 f   libsetlocal001.obj
 0001:000020b4       startAgentThreadWrapper    00000001800030b4 f   libsetlocal001.obj
 0001:000023f4       syncDebuggeeStatus         00000001800033f4 f   libsetlocal001.obj
 0001:00002694       capture_previous_context   0000000180003694 f   MSVCRT:gs_report.obj
 0001:00002708       ?__scrt_initialize_thread_safe_statics@@YAHXZ 0000000180003708 f   MSVCRT:thread_safe_statics.obj
 0001:000027d8       ?__scrt_uninitialize_thread_safe_statics@@YAXXZ 00000001800037d8 f   MSVCRT:thread_safe_statics.obj
 0001:00002880       $$000000                   0000000180003880     MSVCRT:amdsecgs.obj
 0001:000028b0       ?dllmain_crt_dispatch@@YAHQEAUHINSTANCE__@@KQEAX@Z 00000001800038b0 f   MSVCRT:dll_dllmain.obj
 0001:00002900       ?dllmain_crt_process_attach@@YAHQEAUHINSTANCE__@@QEAX@Z 0000000180003900 f   MSVCRT:dll_dllmain.obj
 0001:00002a18       ?dllmain_crt_process_detach@@YAH_N@Z 0000000180003a18 f   MSVCRT:dll_dllmain.obj
 0001:00002a9c       ?dllmain_dispatch@@YAHQEAUHINSTANCE__@@KQEAX@Z 0000000180003a9c f   MSVCRT:dll_dllmain.obj
 0001:000034b0       $$000000                   00000001800044b0     MSVCRT:guard_dispatch.obj
 0001:000034d0       $$000000                   00000001800044d0     MSVCRT:guard_xfg_dispatch.obj
 0001:000034e6       ?fin$0@?0??dllmain_crt_process_attach@@YAHQEAUHINSTANCE__@@QEAX@Z@4HA 00000001800044e6 f   MSVCRT:dll_dllmain.obj
 0001:000034fd       ?fin$0@?0??dllmain_crt_process_detach@@YAH_N@Z@4HA 00000001800044fd f   MSVCRT:dll_dllmain.obj
 0001:00003516       ?fin$1@?0??dllmain_crt_process_detach@@YAH_N@Z@4HA 0000000180004516 f   MSVCRT:dll_dllmain.obj
 0001:0000352a       ?filt$0@?0??dllmain_dispatch@@YAHQEAUHINSTANCE__@@KQEAX@Z@4HA 000000018000452a f   MSVCRT:dll_dllmain.obj
 0001:00003560       __scrt_is_nonwritable_in_current_image$filt$0 0000000180004560 f   MSVCRT:utility.obj
 0002:000001e8       ?__scrt_initialize_tss_var@@3P6AHXZEA 00000001800051e8     MSVCRT:thread_safe_statics.obj
 0002:00000310       ?opcLengths@@3QBEB         0000000180005310     libsetlocal001.obj
 0002:00001da8       GS_ExceptionPointers       0000000180006da8     MSVCRT:gs_report.obj
 0002:00002498       $unwind$fprintf            0000000180007498     libsetlocal001.obj
 0002:000024a4       $unwind$printf             00000001800074a4     libsetlocal001.obj
 0002:000024b0       $unwind$?NewObject@JNIEnv_@@QEAAPEAV_jobject@@PEAV_jclass@@PEAU_jmethodID@@ZZ 00000001800074b0     libsetlocal001.obj
 0002:000024b0       $unwind$nsk_lcomplain      00000001800074b0     libsetlocal001.obj
 0002:000024b0       $unwind$nsk_ldisplay       00000001800074b0     libsetlocal001.obj
 0002:000024b8       $unwind$nsk_lvdisplay      00000001800074b8     libsetlocal001.obj
 0002:000024b8       $unwind$_RTC_Initialize    00000001800074b8     MSVCRT:initsect.obj
 0002:000024b8       $unwind$_RTC_Terminate     00000001800074b8     MSVCRT:initsect.obj
 0002:000024b8       $unwind$?__scrt_initialize_thread_safe_statics@@YAHXZ 00000001800074b8     MSVCRT:thread_safe_statics.obj
 0002:000024c4       $unwind$nsk_lvcomplain     00000001800074c4     libsetlocal001.obj
 0002:000024dc       $unwind$nsk_ltrace         00000001800074dc     libsetlocal001.obj
 0002:000024dc       $unwind$__report_gsfailure 00000001800074dc     MSVCRT:gs_report.obj
 0002:000024e4       $unwind$Agent_Initialize   00000001800074e4     libsetlocal001.obj
 0002:000024e4       $unwind$nsk_lvtrace        00000001800074e4     libsetlocal001.obj
 0002:000024e4       $unwind$__raise_securityfailure 00000001800074e4     MSVCRT:gs_report.obj
 0002:000024e4       $unwind$__scrt_initialize_crt 00000001800074e4     MSVCRT:utility.obj
 0002:000024e4       $unwind$__scrt_initialize_onexit_tables 00000001800074e4     MSVCRT:utility.obj
 0002:000024e4       $unwind$__scrt_release_startup_lock 00000001800074e4     MSVCRT:utility.obj
 0002:000024e4       $unwind$__scrt_uninitialize_crt 00000001800074e4     MSVCRT:utility.obj
 0002:000024e4       $unwind$_onexit            00000001800074e4     MSVCRT:utility.obj
 0002:000024ec       $unwind$nsk_lverify        00000001800074ec     libsetlocal001.obj
 0002:000024fc       $unwind$nsk_vprintf        00000001800074fc     libsetlocal001.obj
 0002:0000250c       $unwind$nsk_printf         000000018000750c     libsetlocal001.obj
 0002:00002514       $unwind$?nsk_jni_lverify@@YAHHPEAUJNIEnv_@@HQEBDH1ZZ 0000000180007514     libsetlocal001.obj
 0002:00002528       $unwind$?nsk_jni_check_exception@@YAHPEAUJNIEnv_@@QEBDH@Z 0000000180007528     libsetlocal001.obj
 0002:00002544       $unwind$Java_nsk_jvmti_unit_FollowReferences_FollowRefObjects_resetTags 0000000180007544     libsetlocal001.obj
 0002:00002544       $unwind$addRefToVerify     0000000180007544     libsetlocal001.obj
 0002:00002544       $unwind$nsk_jvmti_resetAgentData 0000000180007544     libsetlocal001.obj
 0002:00002544       $unwind$nsk_jvmti_setFailStatus 0000000180007544     libsetlocal001.obj
 0002:00002544       $unwind$__scrt_initialize_default_local_stdio_options 0000000180007544     MSVCRT:default_local_stdio_options.obj
 0002:00002544       $unwind$?dllmain_crt_dispatch@@YAHQEAUHINSTANCE__@@KQEAX@Z 0000000180007544     MSVCRT:dll_dllmain.obj
 0002:00002544       $unwind$DllMain            0000000180007544     MSVCRT:dll_dllmain_stub.obj
 0002:00002544       $unwind$__GSHandlerCheck   0000000180007544     MSVCRT:gshandler.obj
 0002:00002544       $unwind$?__scrt_uninitialize_thread_safe_statics@@YAXXZ 0000000180007544     MSVCRT:thread_safe_statics.obj
 0002:00002544       $unwind$__scrt_acquire_startup_lock 0000000180007544     MSVCRT:utility.obj
 0002:00002544       $unwind$__scrt_dllmain_after_initialize_c 0000000180007544     MSVCRT:utility.obj
 0002:00002544       $unwind$__scrt_dllmain_before_initialize_c 0000000180007544     MSVCRT:utility.obj
 0002:00002544       $unwind$__scrt_dllmain_crt_thread_attach 0000000180007544     MSVCRT:utility.obj
 0002:00002544       $unwind$__scrt_dllmain_crt_thread_detach 0000000180007544     MSVCRT:utility.obj
 0002:00002544       $unwind$__scrt_dllmain_uninitialize_c 0000000180007544     MSVCRT:utility.obj
 0002:00002544       $unwind$__scrt_dllmain_uninitialize_critical 0000000180007544     MSVCRT:utility.obj
 0002:00002544       $unwind$atexit             0000000180007544     MSVCRT:utility.obj
 0002:0000254c       $unwind$nsk_jvmti_lverify  000000018000754c     libsetlocal001.obj
 0002:00002560       $unwind$exitOnError        0000000180007560     libsetlocal001.obj
 0002:00002570       $unwind$Java_nsk_share_jvmti_ArgumentHandler_getAgentOptionsString 0000000180007570     libsetlocal001.obj
 0002:00002584       $unwind$Java_nsk_jvmti_unit_FollowReferences_FollowRefObjects_getTag 0000000180007584     libsetlocal001.obj
 0002:00002584       $unwind$Java_nsk_share_jvmti_DebugeeClass_checkStatus 0000000180007584     libsetlocal001.obj
 0002:00002584       $unwind$agentThreadWrapper 0000000180007584     libsetlocal001.obj
 0002:00002594       $unwind$startAgentThreadWrapper 0000000180007594     libsetlocal001.obj
 0002:000025b0       $unwind$syncDebuggeeStatus 00000001800075b0     libsetlocal001.obj
 0002:000025b0       $unwind$__scrt_dllmain_exception_filter 00000001800075b0     MSVCRT:utility.obj
 0002:000025c4       $unwind$Java_nsk_share_jvmti_DebugeeClass_resetAgentData 00000001800075c4     libsetlocal001.obj
 0002:000025cc       $unwind$MA_checkStatus     00000001800075cc     libsetlocal001.obj
 0002:000025e0       $unwind$Java_nsk_jvmti_unit_FollowReferences_FollowRefObjects_setTag 00000001800075e0     libsetlocal001.obj
 0002:000025f8       $unwind$Java_nsk_jvmti_unit_FollowReferences_FollowRefObjects_addRefToVerify 00000001800075f8     libsetlocal001.obj
 0002:00002614       $unwind$check_error        0000000180007614     libsetlocal001.obj
 0002:00002620       $unwind$Breakpoint         0000000180007620     libsetlocal001.obj
 0002:00002638       $unwind$Java_nsk_jvmti_SetLocalVariable_setlocal001_getMethReady 0000000180007638     libsetlocal001.obj
 0002:00002650       $unwind$capture_previous_context 0000000180007650     MSVCRT:gs_report.obj
 0002:0000265c       $unwind$__GSHandlerCheckCommon 000000018000765c     MSVCRT:gshandler.obj
 0002:00002668       $xdatasym                  0000000180007668     MSVCRT:amdsecgs.obj
 0002:0000266c       $unwind$?dllmain_crt_process_attach@@YAHQEAUHINSTANCE__@@QEAX@Z 000000018000766c     MSVCRT:dll_dllmain.obj
 0002:000026a8       $unwind$?fin$0@?0??dllmain_crt_process_attach@@YAHQEAUHINSTANCE__@@QEAX@Z@4HA 00000001800076a8     MSVCRT:dll_dllmain.obj
 0002:000026a8       $unwind$?fin$0@?0??dllmain_crt_process_detach@@YAH_N@Z@4HA 00000001800076a8     MSVCRT:dll_dllmain.obj
 0002:000026a8       $unwind$?fin$1@?0??dllmain_crt_process_detach@@YAH_N@Z@4HA 00000001800076a8     MSVCRT:dll_dllmain.obj
 0002:000026b0       $unwind$?dllmain_crt_process_detach@@YAH_N@Z 00000001800076b0     MSVCRT:dll_dllmain.obj
 0002:00002704       $unwind$?dllmain_dispatch@@YAHQEAUHINSTANCE__@@KQEAX@Z 0000000180007704     MSVCRT:dll_dllmain.obj
 0002:0000272c       $unwind$?filt$0@?0??dllmain_dispatch@@YAHQEAUHINSTANCE__@@KQEAX@Z@4HA 000000018000772c     MSVCRT:dll_dllmain.obj
 0002:00002734       $unwind$_DllMainCRTStartup 0000000180007734     MSVCRT:dll_dllmain.obj
 0002:00002744       $unwind$__scrt_is_nonwritable_in_current_image 0000000180007744     MSVCRT:utility.obj
 0002:00002764       $unwind$__scrt_is_nonwritable_in_current_image$filt$0 0000000180007764     MSVCRT:utility.obj
 0002:0000276c       $unwind$__scrt_fastfail    000000018000776c     MSVCRT:utility_desktop.obj
 0002:0000277c       $unwind$__security_init_cookie 000000018000777c     MSVCRT:gs_support.obj
 0002:00002788       $unwind$__isa_available_init 0000000180007788     MSVCRT:cpu_disp.obj
 0002:00002798       $xdatasym                  0000000180007798     MSVCRT:guard_dispatch.obj
 0002:000027a0       $xdatasym                  00000001800077a0     MSVCRT:guard_xfg_dispatch.obj
 0002:000027b0       .edata                     00000001800077b0     setlocal001.exp
 0002:000027d8       rgpv                       00000001800077d8     setlocal001.exp
 0002:00002818       rgszName                   0000000180007818     setlocal001.exp
 0002:00002858       rgwOrd                     0000000180007858     setlocal001.exp
 0002:00002878       szName                     0000000180007878     setlocal001.exp
 0002:00002888       $N00001                    0000000180007888     setlocal001.exp
 0002:00002897       $N00002                    0000000180007897     setlocal001.exp
 0002:000028a4       $N00003                    00000001800078a4     setlocal001.exp
 0002:000028dd       $N00004                    00000001800078dd     setlocal001.exp
 0002:00002910       $N00005                    0000000180007910     setlocal001.exp
 0002:00002955       $N00006                    0000000180007955     setlocal001.exp
 0002:00002992       $N00007                    0000000180007992     setlocal001.exp
 0002:000029da       $N00008                    00000001800079da     setlocal001.exp
 0002:00002a1a       $N00009                    0000000180007a1a     setlocal001.exp
 0002:00002a57       $N00010                    0000000180007a57     setlocal001.exp
 0002:00002a92       $N00011                    0000000180007a92     setlocal001.exp
 0002:00002ac0       $N00012                    0000000180007ac0     setlocal001.exp
 0002:00002af1       $N00013                    0000000180007af1     setlocal001.exp
 0002:00002b20       $N00014                    0000000180007b20     setlocal001.exp
 0002:00002b4f       $N00015                    0000000180007b4f     setlocal001.exp
 0002:00002b84       $N00016                    0000000180007b84     setlocal001.exp
 0002:00002f92       .idata$6                   0000000180007f92     kernel32:KERNEL32.dll
 0002:00002ff6       .idata$6                   0000000180007ff6     vcruntime:VCRUNTIME140.dll
 0002:00003162       .idata$6                   0000000180008162     ucrt:api-ms-win-crt-runtime-l1-1-0.dll
 0002:00003184       .idata$6                   0000000180008184     ucrt:api-ms-win-crt-stdio-l1-1-0.dll
 0002:000031a4       .idata$6                   00000001800081a4     ucrt:api-ms-win-crt-string-l1-1-0.dll
 0003:00000000       ?codeAttributeName@@3PEBDEB 0000000180009000     libsetlocal001.obj
 0003:00000008       ?lineNumberAttributeName@@3PEBDEB 0000000180009008     libsetlocal001.obj
 0003:00000010       ?localVarAttributeName@@3PEBDEB 0000000180009010     libsetlocal001.obj
 0003:00000018       ?localVarTypeAttributeName@@3PEBDEB 0000000180009018     libsetlocal001.obj
 0003:00000020       ?stackMapAttributeName@@3PEBDEB 0000000180009020     libsetlocal001.obj
 0003:00000028       ?callBytes@@3PAEA          0000000180009028     libsetlocal001.obj
 0003:0000002c       ?allocBytes@@3PAEA         000000018000902c     libsetlocal001.obj
 0003:00000030       longVal                    0000000180009030     libsetlocal001.obj
 0003:0001aad4       redefineAttempted          0000000180023ad4     libsetlocal001.obj
 0003:0001aad8       nsk_context                0000000180023ad8     libsetlocal001.obj
 0003:0001aae4       redefineSucceed            0000000180023ae4     libsetlocal001.obj
 0003:0001aae8       agentFailed                0000000180023ae8     libsetlocal001.obj
 0003:0001aaec       currentAgentStatus         0000000180023aec     libsetlocal001.obj
 0003:0001aaf0       context                    0000000180023af0     libsetlocal001.obj
 0003:0001aba8       agentThread                0000000180023ba8     libsetlocal001.obj
 0003:0001abb0       agentThreadProc            0000000180023bb0     libsetlocal001.obj
 0003:0001abb8       agentThreadArg             0000000180023bb8     libsetlocal001.obj
 0003:0001abc0       agent_data                 0000000180023bc0     libsetlocal001.obj
 0003:0001abd0       jvmti_env                  0000000180023bd0     libsetlocal001.obj
 0003:0001abd8       jvm                        0000000180023bd8     libsetlocal001.obj
 0003:0001abe0       jni_env                    0000000180023be0     libsetlocal001.obj
 0003:0001abe8       checkStatus_func           0000000180023be8     libsetlocal001.obj
 0003:0001abf0       ?codeAttributeIndex@@3GA   0000000180023bf0     libsetlocal001.obj
 0003:0001abf4       ?lineNumberAttributeIndex@@3GA 0000000180023bf4     libsetlocal001.obj
 0003:0001abf8       ?localVarAttributeIndex@@3GA 0000000180023bf8     libsetlocal001.obj
 0003:0001abfc       ?localVarTypeAttributeIndex@@3GA 0000000180023bfc     libsetlocal001.obj
 0003:0001ac00       ?stackMapAttributeIndex@@3GA 0000000180023c00     libsetlocal001.obj
 0003:0001ac04       ?stackFrameOffset@@3GA     0000000180023c04     libsetlocal001.obj
 0003:0001ac08       ?mode@@3HA                 0000000180023c08     libsetlocal001.obj
 0003:0001ac0c       ?constantPoolSize@@3GA     0000000180023c0c     libsetlocal001.obj
 0003:0001ac10       ?orig@@3PEBEEB             0000000180023c10     libsetlocal001.obj
 0003:0001ac18       ?gen@@3PEAEEA              0000000180023c18     libsetlocal001.obj
 0003:0001ac20       ?inputPos@@3PEAEEA         0000000180023c20     libsetlocal001.obj
 0003:0001ac28       ?endPos@@3PEBEEB           0000000180023c28     libsetlocal001.obj
 0003:0001ac30       ?genPos@@3PEAEEA           0000000180023c30     libsetlocal001.obj
 0003:0001ac38       ?markPos@@3PEAEEA          0000000180023c38     libsetlocal001.obj
 0003:0001ac40       ?constantPool@@3PEAPEADEA  0000000180023c40     libsetlocal001.obj
 0003:0001ac48       ?constantPoolCount@@3GA    0000000180023c48     libsetlocal001.obj
 0003:0001ac4c       ?zeroBytes@@3PAEA          0000000180023c4c     libsetlocal001.obj
 0003:0001ac50       ?codeLength@@3IA           0000000180023c50     libsetlocal001.obj
 0003:0001ac54       result                     0000000180023c54     libsetlocal001.obj
 0003:0001ac58       ?map@@3PEAIEA              0000000180023c58     libsetlocal001.obj
 0003:0001ac60       ?widening@@3PEACEA         0000000180023c60     libsetlocal001.obj
 0003:0001ac68       jvmti                      0000000180023c68     libsetlocal001.obj
 0003:0001ac70       caps                       0000000180023c70     libsetlocal001.obj
 0003:0001ac80       callbacks                  0000000180023c80     libsetlocal001.obj
 0003:0001adb8       mid1                       0000000180023db8     libsetlocal001.obj
 0003:0001adc0       mid2                       0000000180023dc0     libsetlocal001.obj
 0003:0001adc8       mid3                       0000000180023dc8     libsetlocal001.obj
 0003:0001add0       mid4                       0000000180023dd0     libsetlocal001.obj
 0003:0001add8       floatVal                   0000000180023dd8     libsetlocal001.obj
 0003:0001ade0       doubleVal                  0000000180023de0     libsetlocal001.obj
 0003:0001ade8       objVal                     0000000180023de8     libsetlocal001.obj
 0003:0001adf0       arrVal                     0000000180023df0     libsetlocal001.obj
 0003:0001ae00       GS_ExceptionRecord         0000000180023e00     MSVCRT:gs_report.obj
 0003:0001aea0       GS_ContextRecord           0000000180023ea0     MSVCRT:gs_report.obj
 0003:0001b370       ?g_tss_cv@@3U_RTL_CONDITION_VARIABLE@@A 0000000180024370     MSVCRT:thread_safe_statics.obj
 0003:0001b378       ?g_tss_event@@3PEAXEA      0000000180024378     MSVCRT:thread_safe_statics.obj
 0003:0001b380       ?g_tss_mutex@@3U_RTL_CRITICAL_SECTION@@A 0000000180024380     MSVCRT:thread_safe_statics.obj
 0003:0001b3a8       ?g_sleep_condition_variable_cs@@3P6AHPEAU_RTL_CONDITION_VARIABLE@@PEAU_RTL_CRITICAL_SECTION@@K@ZEA 00000001800243a8     MSVCRT:thread_safe_statics.obj
 0003:0001b3b0       ?g_wake_all_condition_variable@@3P6AXPEAU_RTL_CONDITION_VARIABLE@@@ZEA 00000001800243b0     MSVCRT:thread_safe_statics.obj
 0003:0001b3bc       ?__proc_attached@@3HA      00000001800243bc     MSVCRT:dll_dllmain.obj
 0003:0001b3d0       ?is_initialized_as_dll@@3_NA 00000001800243d0     MSVCRT:utility.obj
 0003:0001b3d1       ?module_local_atexit_table_initialized@@3_NA 00000001800243d1     MSVCRT:utility.obj
 0003:0001b3d8       ?module_local_atexit_table@@3U_onexit_table_t@@A 00000001800243d8     MSVCRT:utility.obj
 0003:0001b3f0       ?module_local_at_quick_exit_table@@3U_onexit_table_t@@A 00000001800243f0     MSVCRT:utility.obj
